:1000000002C1000049C600001CC60000EFC5000088
:10001000C2C5000095C5000068C5000024C10000ED
:1000200022C1000020C100001EC100001CC1000050
:100030001AC1000018C1000016C1000014C1000060
:1000400012C1000010C100000EC100000CC1000070
:100050000AC1000008C1000006C10000FCC4000085
:1000600002C10000C2C4000097C40000FCC0000030
:10007000FAC00000F8C00000F6C00000F4C00000A4
:10008000F2C00000F0C00000EEC00000ECC00000B4
:10009000EAC00000E8C00000E6C00000E4C00000C4
:1000A000E2C00000E0C00000DEC00000DCC00000D4
:1000B000DAC00000D8C00000D6C00000D4C00000E4
:1000C000D2C00000D0C00000CEC00000CCC00000F4
:1000D000CAC00000C8C00000C6C00000C4C0000004
:1000E000C2C0000000002100240027002A002D00CB
:1000F0003000330001010000040107010A01000083
:100100002200250028002B002E00310034000201BF
:100110000000050108010B0100000A0B02090C0D8B
:100120000E080703040100000000000000000000AA
:1001300000000000000000000000000000000000BF
:10014000000000001211100000000000000000007C
:10015000000000000000000000000000000001029C
:1001600010202008081020401020408002010201C9
:100170000804020101020408102040808040201081
:1001800008040201800402018040201008040201DA
:100190000804020101020408102040800102040842
:1001A00010204080000020002300260029002C00A1
:1001B0002F003200000100000301060109010505BE
:1001C0000505070508080808020202020A0A0808CD
:1001D00004040404010101010101010103030303FB
:1001E00003030303040707070C0C0C0C0C0C0C0C8A
:1001F0000202020206060606060606060B0B0B0B9B
:100200000B0B0B0BD90611241FBECFEFD1E2DEBFC3
:10021000CDBF00E00CBF25E0A2EAB3E001C01D9213
:10022000AC38B207E1F713E0A0E0B2E0E2EAF9E1AE
:1002300000E00BBF02C007900D92A23AB107D9F7B8
:1002400011E0C3E0D1E000E006C021970109802F52
:10025000FE010E949E0BC230D10780E00807A9F77B
:100260005FD60C94CF0CCCCEAF92BF92CF92DF92E0
:10027000EF92FF920F931F93CF93DF936C017B015B
:100280008B01040F151FEB015E01AE18BF08C017EC
:10029000D10759F06991D601ED91FC910190F0815F
:1002A000E02DC6011995892B79F7C501DF91CF9112
:1002B0001F910F91FF90EF90DF90CF90BF90AF9084
:1002C0000895FC01538D448D252F30E0842F90E05C
:1002D000821B930B541710F0CF9608950197089541
:1002E000FC01918D828D981761F0A28DAE0FBF2F0A
:1002F000B11D5D968C91928D9F5F9F73928F90E060
:1003000008958FEF9FEF0895FC01918D828D9817CE
:1003100031F0828DE80FF11D858D90E008958FEF0B
:100320009FEF0895FC01918D228D892F90E0805CD4
:100330009F4F821B91098F73992708958BE194E059
:10034000F1DF21E0892B09F420E0822F0895FC01E0
:10035000A48DA80FB92FB11DA35ABF4F2C91848D26
:1003600090E001968F739927848FA689B7892C9383
:10037000A089B1898C91837080648C93938D848DD6
:10038000981306C00288F389E02D80818F7D8083D9
:100390000895EF92FF920F931F93CF93DF93EC0199
:1003A00081E0888F9B8D8C8D98131AC0E889F9891C
:1003B000808185FF15C09FB7F894EE89FF8960831F
:1003C000E889F98980818370806480839FBF81E0A0
:1003D00090E0DF91CF911F910F91FF90EF900895E2
:1003E000F62E0B8D10E00F5F1F4F0F731127E02EBD
:1003F0008C8D8E110BC00FB607FCFACFE889F989F6
:10040000808185FFF5CFCE01A2DFF2CFEB8DEC0F1F
:10041000FD2FF11DE35AFF4FF0829FB7F8940B8F29
:10042000EA89FB8980818062D0CFCF93DF93EC0192
:10043000888D8823B1F0AA89BB89E889F9898C91D4
:1004400085FD03C0808186FD0CC00FB607FCF7CF89
:100450008C9185FFF2CF808185FFEDCFCE0177DFD4
:10046000EACFDF91CF9108958150823108F05AC0D0
:10047000E82FF0E08827E05CFD4F8F4F0C949E0B37
:1004800060026402520258025C02920267026D022C
:10049000710277027B027F028502890292028D023D
:1004A00093029702809180008F7780938000089557
:1004B000809180008F7DF9CF80918000877FF5CF7C
:1004C00084B58F7784BD089584B58F7DFBCF8091EF
:1004D000B0008F778093B00008958091B0008F7D39
:1004E000F9CF809190008F7780939000089580914C
:1004F00090008F7DF9CF80919000877FF5CF80911C
:10050000A0008F778093A00008958091A0008F7D38
:10051000F9CF8091A000877FF5CF809120018F7760
:10052000809320010895809120018F7DF9CF8091E3
:100530002001877FF5CF1F93CF93DF93282F30E0E3
:10054000F901E85EFE4F8491F901E25AFE4FD49121
:10055000F901E254FE4FC491CC23A1F0162F811172
:1005600083DFEC2FF0E0EE0FFF1FE250FF4FA5916D
:10057000B4918FB7F894EC91111108C0D095DE2397
:10058000DC938FBFDF91CF911F910895DE2BF8CFC1
:10059000CF93DF9390E0FC01E25AFE4F2491825406
:1005A0009E4FFC0184918823C9F090E0880F991F29
:1005B000FC01EC51FF4FA591B491FC01E250FF4FBB
:1005C000C591D49161110DC09FB7F8948C9120957D
:1005D00082238C938881282328839FBFDF91CF912A
:1005E0000895623051F49FB7F8943C91822F809522
:1005F00083238C93E8812E2BEFCF8FB7F894EC9167
:100600002E2B2C938FBFEACF3FB7F89480910D0427
:1006100090910E04A0910F04B091100426B5A89BF0
:1006200005C02F3F19F00196A11DB11D3FBFBA2F84
:10063000A92F982F8827BC01CD01620F711D811D44
:10064000911D42E0660F771F881F991F4A95D1F7C9
:1006500008958F929F92AF92BF92CF92DF92EF92C6
:10066000FF924B015C01D0DF6B017C01CDDF6C1987
:100670007D098E099F09683E734081059105B0F39D
:1006800021E0821A9108A108B10888EEC80E83E023
:10069000D81EE11CF11C81149104A104B10431F7AE
:1006A000FF90EF90DF90CF90BF90AF909F908F9092
:1006B00008952FB7F8946091090470910A0480910D
:1006C0000B0490910C042FBF0895FC01848187FDD9
:1006D00004C091E0692763832EDF80E00895FC0168
:1006E000808580FD04C082FB882780F9089580E022
:1006F0000895FC019085957081E0953009F080E0C7
:100700000895862F642F44CFCF93DF93FC0121857A
:1007100030E0F901E85EFE4F8491F901E25AFE4FA4
:10072000D491F901E254FE4FC491CC2371F08111B0
:100730009BDEEC2FF0E0EE0FFF1FEC55FE4FA59176
:10074000B491EC91ED2381E009F480E08170DF91B8
:10075000CF9108950F931F93CF93DF938BE194E094
:10076000E1DD892BA1F18BE194E0BADD8C3329F432
:100770001092070410920604F1CF8A30B1F4C0E25F
:10078000D2E002EA13E089919991009739F0F801DB
:10079000208161E0213309F060E0CDDE0F5F1F4F63
:1007A000F2E0C633DF0779F7E3CF209106043091FA
:1007B000070424363105E4F6F901EE55FC4F808339
:1007C0002F5F3F4F3093070420930604C7CFDF917C
:1007D000CF911F910F910895B1DD8111BBDF80E0B2
:1007E00090E0892B49F080E090E0892B29F00E946D
:1007F000000081110E94000080E090E0892B49F008
:1008000080E090E0892B29F00E94000081110E9475
:10081000000080E090E0892B49F080E090E0892B97
:1008200029F00E94000081110C9400000895DC0161
:10083000ED91FD918081ED91FD919081ED91FD9182
:100840006C9163708E2309F064609F2309F06860E7
:10085000E4E3F4E0E60FF11D659565956D936D9108
:100860007D918D919D91099423C01AC012C016C02C
:1008700010C01EC009C014C013C006C019C009C0F2
:100880000DC007C00DC014C0625070408040904041
:100890000BC0615070408040904006C06E5F01C048
:1008A0006F5F7F4F8F4F9F4F9E938E937E936E937C
:1008B000089580916905823070F4F8948EE595E092
:1008C000B6DF60916505709166058091670590912E
:1008D000680578940895F894F4CF8F929F92AF9220
:1008E000BF920F931F93CF93DF93CDB7DEB7A1973E
:1008F0000FB6F894DEBF0FBECDBF19A2423008F488
:100900004AE08E010F5D1F4F842E912CB12CA12C3B
:10091000A5019401D5D6E62FB901CA01EA303CF50C
:10092000E05DD801EE938D01232B242B252B81F73D
:1009300090E080E0109761F0FD0101900020E9F760
:100940003197AF014A1B5B0BBD018BE194E08CDC5E
:10095000A1960FB6F894DEBF0FBECDBFDF91CF9149
:100960001F910F91BF90AF909F908F900895E95C79
:10097000D8CF009761F0FC0101900020E9F7319792
:10098000AF01481B590BBC018BE194E06DCC90E0AA
:1009900080E008950E94CB0C1F920F920FB60F9229
:1009A00011240BB60F922F933F934F935F936F9346
:1009B0007F938F939F93AF93BF93EF93FF938BE1BD
:1009C00094E0C5DCFF91EF91BF91AF919F918F9122
:1009D0007F916F915F914F913F912F910F900BBE3F
:1009E0000F900FBE0F901F9018951F920F920FB689
:1009F0000F9211240BB60F922F938F939F93EF9327
:100A0000FF93E0912B04F0912C048081E09131045C
:100A1000F091320482FD1DC09081809134048F5F7B
:100A20008F7320913504821741F0E0913404F0E097
:100A3000E55EFB4F958F80933404FF91EF919F917A
:100A40008F912F910F900BBE0F900FBE0F901F90A4
:100A500018958081F2CF1F920F920FB60F9211243A
:100A60002F933F938F939F93AF93BF9380910904EC
:100A700090910A04A0910B04B0910C0430910804E9
:100A800023E0230F2D3758F50196A11DB11D2093AA
:100A900008048093090490930A04A0930B04B09374
:100AA0000C0480910D0490910E04A0910F04B0915C
:100AB00010040196A11DB11D80930D0490930E04A6
:100AC000A0930F04B0931004BF91AF919F918F91A9
:100AD0003F912F910F900FBE0F901F90189526E811
:100AE000230F0296A11DB11DD2CF1F920F920FB6F8
:100AF0000F9211240BB60F922F933F934F935F9356
:100B00006F937F938F939F93AF93BF93EF93FF93D5
:100B10008091BA049091BB048ADEFF91EF91BF915E
:100B2000AF919F918F917F916F915F914F913F9185
:100B30002F910F900BBE0F900FBE0F901F90189526
:100B40001F920F920FB60F9211240BB60F922F9394
:100B50003F934F935F936F937F938F939F93AF9345
:100B6000BF93EF93FF938091B8049091B9045FDE37
:100B7000FF91EF91BF91AF919F918F917F916F9175
:100B80005F914F913F912F910F900BBE0F900FBE31
:100B90000F901F9018951F920F920FB60F9211246D
:100BA0000BB60F922F933F934F935F936F937F9367
:100BB0008F939F93AF93BF93EF93FF938091C20462
:100BC0009091C30434DEFF91EF91BF91AF919F915B
:100BD0008F917F916F915F914F913F912F910F90E6
:100BE0000BBE0F900FBE0F901F9018951F920F9283
:100BF0000FB60F9211240BB60F922F933F934F9382
:100C00005F936F937F938F939F93AF93BF93EF9374
:100C1000FF938091C0049091C10409DEFF91EF9190
:100C2000BF91AF919F918F917F916F915F914F9104
:100C30003F912F910F900BBE0F900FBE0F901F9002
:100C400018951F920F920FB60F9211240BB60F92A8
:100C50002F933F934F935F936F937F938F939F93C4
:100C6000AF93BF93EF93FF938091BE049091BF0425
:100C7000DEDDFF91EF91BF91AF919F918F917F91B9
:100C80006F915F914F913F912F910F900BBE0F90FD
:100C90000FBE0F901F9018951F920F920FB60F92D4
:100CA00011240BB60F922F933F934F935F936F9343
:100CB0007F938F939F93AF93BF93EF93FF93809115
:100CC000BC049091BD04B3DDFF91EF91BF91AF9152
:100CD0009F918F917F916F915F914F913F912F9154
:100CE0000F900BBE0F900FBE0F901F901895CF92D4
:100CF000DF92EF92FF920F931F93CF93DF93EC015C
:100D0000E62E84E090E022D5FC0184E6808385E62F
:100D1000818386E6828387E6838386E692E09983F1
:100D200088838FEF8A838B838C838A878B878C87DA
:100D300084E089878F016E0185E0C80ED11CF12CFB
:100D4000F80181918F0187FD32C0F60181936F0117
:100D500061E01EDCF394F4E0FF12F2CF8FEF8C839E
:100D60008CE692E0998388838B8587FD0FC0282FBE
:100D7000082E000C330BE216130641F09A859130D1
:100D800011F460E0D8DB60E08B8502DC82E08A87CA
:100D9000EB8662E08E2DFCDB81E08C87DF91CF91CA
:100DA0001F910F91FF90EF90DF90CF900895F986FB
:100DB000D5CFCF93DF9310921E0410921D0488EEBE
:100DC00093E0A0E0B0E080931F0490932004A093F0
:100DD0002104B093220482E792E090931C04809354
:100DE0001B0485EC90E0909328048093270484EC06
:100DF00090E090932A048093290480EC90E09093F3
:100E00002C0480932B0481EC90E090932E0480932B
:100E10002D0482EC90E09093300480932F0486ECB4
:100E200090E0909332048093310410923404109235
:100E30003504109236041092370462E68BE795E091
:100E400056DF63E68EE695E052DF62E087E2A0DBE4
:100E500062E081E39DDBE5EEF1E0E491F0E0EE0F8E
:100E6000FF1FEC55FE4FA591B491B0935F05A09381
:100E70005E05E5E8F1E0449140936205EFEEF1E0B4
:100E8000E491F0E0EE0FFF1FEC55FE4FC591D491B9
:100E9000D0936105C0936005EFE8F1E0E491E09341
:100EA0006305109265051092660510926705109211
:100EB00068052BE33FE1C9010197F1F79C91842F6D
:100EC000892391E009F490E08881E82309F0926099
:100ED000909364051092690588E892E090936B0501
:100EE00080936A0585E992E090936D0580936C0587
:100EF000E4ECF4E024E832E08AE090E031832083FF
:100F0000128213821482158297838683108611863B
:100F10003E9645E0EE35F40789F7DF91CF910895CD
:100F2000CF93DF9300D01F92CDB7DEB7789484B50E
:100F3000826084BD84B5816084BD85B5826085BDD5
:100F400085B5816085BD80916E00816080936E0063
:100F50001092810080918100826080938100809155
:100F60008100816080938100809180008160809306
:100F700080008091B10084608093B1008091B000C6
:100F800081608093B0008091910082608093910095
:100F900080919100816080939100809190008160A8
:100FA000809390008091A10082608093A100809145
:100FB000A10081608093A1008091A0008160809356
:100FC000A000809121018260809321018091210104
:100FD00081608093210180912001816080932001B4
:100FE00080917A00846080937A0080917A00826098
:100FF00080937A0080917A00816080937A0080915A
:101000007A00806880937A001092C1006EE5C62E47
:1010100065E0D62E24EC34E03C832B8306E312E01B
:101020007AE0A72EB12CD801FC9011967C91AB816F
:10103000BC81ED91FC9111970280F381E02D42E09B
:1010400050E06F2DCD011995EB81FC81F186108662
:10105000DF010190F081E02D0190F081E02DCD01C4
:101060001995882329F0EB81FC8180858360808736
:1010700020DBAB81BC8112966D937D938D939C9305
:1010800015971796BC92AE9216970C5F1F4F1E963F
:10109000BC83AB83CA16DB0631F60BDC6093170406
:1010A000709318048093190490931A0400E212E0DC
:1010B00056E3C52E52E0D52E1C830B83AB81BC8139
:1010C000ED90FD90BC83AB83E114F10431F061E05D
:1010D0008E2D5EDA61E08E2D2EDA2B803C80C214DC
:1010E000D30461F768E873E180E090E0B2DAD801F8
:1010F0008D919D918D01009711F060E01CDA2B809D
:101100003C800215130599F7E0912B04F0912C0413
:1011100082E08083E0912704F09128041082E0911E
:101120002904F0912A0480E1808310923304E09135
:101130002F04F091300486E08083E0912D04F0913B
:101140002E04808180618083E0912D04F0912E0433
:10115000808188608083E0912D04F0912E0480814D
:1011600080688083E0912D04F0912E0480818F7D32
:10117000808382E390E0A0E0B0E080931F0490932E
:101180002004A0932104B093220482EA92E022E09A
:10119000853B920709F45FC031E039838B5C924054
:1011A00009F0198242EA642E42E0742E82DA4B0181
:1011B0005C018091160290911702A0911802B091E3
:1011C0001902AC01BD014854544F6F4F7F4F841634
:1011D0009506A606B70628F488169906AA06BB0641
:1011E00040F581EE92E0C5DB82EA92E0C2DB80EF5F
:1011F00092E0BFDB4AE064E070E080E090E06DDB0D
:1012000080EF92E0B6DB80E192E0B3DB8CE293E02A
:10121000B0DB8092160290921702A0921802B09250
:10122000190280920C0290920D02A0920E02B092CE
:101230000F02F1E0FA832EE2621623E0720609F053
:101240001A8280916A0590916B0533E0813493078F
:1012500029F421E013C081E08983A4CF825F92400A
:10126000C1F380916C0590916D0521E0B2E08D3F56
:101270009B0721F08850934009F020E02A8022202B
:1012800009F4F0C0222309F4EDC013DB24E030E0C0
:1012900040E050E037D269017A01809117049091C3
:1012A0001804A0911904B0911A048C159D05AE057F
:1012B000BF050CF0DDC080916C0590916D0559DB88
:1012C0008CE293E056DB80920C0290920D02A09289
:1012D0000E02B0920F02C0921704D0921804E0924E
:1012E0001904F0921A0436E3C32E32E0D32E24EC14
:1012F00034E03C832B83F12CE12CAB81BC8118962C
:101300008C9118978B7F18968C931897ED91FC9180
:1013100011970190F081E02DCD011995182FEB81E7
:10132000FC81808586958170181709F4ACC0C1D9FD
:10133000AB81BC8112966D937D938D939C93159791
:1013400018968C91B2E08B27EB81FC8180878B8192
:101350009C81C5D9811106C08B819C81CAD9882303
:1013600009F46FC021E0F3E16F16F3E07F0609F0A6
:1013700020E0D6010D911C91C8010397039708F452
:10138000BDC081E00431110509F080E0222311F095
:10139000811111C0C8014397039708F4B1C081E0DF
:1013A0000C31110509F080E02980222009F4AAC03F
:1013B000882309F4A7C08092080290920902A092A3
:1013C0000A02B0920B021092160410921504D60174
:1013D00012968D919C91CDDA8B819C8180D9882346
:1013E00009F45DC186E293E0C4DA0B321105E1F441
:1013F0002A802220C9F08091110490911204009754
:1014000009F044C144244394512C50921204409258
:1014100011048092000290920102A0920202B09206
:10142000030261E080E087D864E670E080E090E04D
:1014300010D980920C0290920D02A0920E02B092EE
:101440000F022FEFE21AF20A8B819C810E969C8389
:101450008B8394E0C90ED11CABE0EA16F10409F0CD
:101460004CCF81C026DA22E030E040E050E012CFDD
:10147000C816D906EA06FB060CF02DCF80916A0546
:1014800090916B051CCF15D9AB81BC8112962D9123
:101490003D914D915C9115971B012C01221A330A45
:1014A000440A550AB201A10116968D919C91B0E0B3
:1014B000A0E0481759076A077B0708F448CFAB81BB
:1014C000BC8118968C918170181709F440CFF1D81F
:1014D000EB81FC8162837383848395838085F1E053
:1014E0008F278460AB81BC8118968C93E2D8EB8106
:1014F000FC81628773878487958729CF81E046CFF7
:1015000081E052CF0231110511F4211108C00A31D6
:10151000110509F05CCF3980332009F458CF809150
:10152000080290910902A0910A02B0910B02865024
:101530009F4FAF4FBF4F88169906AA06BB0698F07B
:1015400044244394512C5092160440921504F09276
:101550001404E09213048092040290920502A09277
:101560000602B0920702BEE26B16B3E07B0601F5FD
:101570008091000290910102A0910202B0910302B9
:1015800088539D4CAF4FBF4F88159905AA05BB05E1
:1015900020F4109212041092110480911104909181
:1015A000120460E0892B09F061E080E00E949B0258
:1015B00080910C0290910D02A0910E02B0910F0249
:1015C000AC01BD014C595F4F6F4F7F4F841695069C
:1015D000A606B70628F488169906AA06BB0658F48C
:1015E0008CE293E0C6D980920C0290920D02A092F8
:1015F0000E02B0920F028091040290910502A09118
:101600000602B091070286509F4FAF4FBF4F88151B
:101610009905AA05BB05C0F58091150490911604A3
:10162000019791F5E0911304F0911404EE0FFF1F60
:10163000EE0FFF1FEA5CFD4F828193819AD9809162
:10164000130490911404EEE0E89F8001E99F100DCF
:1016500011240C531B4FC80142D8882351F186E254
:1016600093E087D964E670E080E090E00E9429036F
:1016700080920C0290920D02A0920E02B0920F0284
:101680001092160410921504A7D890CD019709F076
:10169000CBCE109212041092110460E0C3CE8B8165
:1016A0009C8127D8882309F4BFCE8AE293E061D9D0
:1016B000BBCEC8011ED88823A9F28AE293E0D1CF1D
:1016C000A1E21A2EAA1BBB1BFD010DC0AA1FBB1F46
:1016D000EE1FFF1FA217B307E407F50720F0A21BB8
:1016E000B30BE40BF50B661F771F881F991F1A9425
:1016F00069F760957095809590959B01AC01BD014F
:10170000CF010895052E97FB16F400940FD057FDD6
:1017100005D0D6DF07FC02D046F408C050954095AE
:10172000309521953F4F4F4F5F4F0895909580958D
:10173000709561957F4F8F4F9F4F0895EE0FFF1F5C
:10174000881F8BBF0790F691E02D19940F931F937C
:10175000CF93DF938230910510F482E090E0E09126
:101760008A05F0918B0530E020E0B0E0A0E03097F2
:1017700099F42115310509F44AC0281B390B24308E
:101780003105D8F58A819B816115710589F1FB01CD
:1017900093838283FE0111C04081518102811381B4
:1017A00048175907E0F04817590799F4109761F066
:1017B00012960C93129713961C933296CF01DF91D9
:1017C000CF911F910F91089500938A0510938B0577
:1017D000F4CF2115310551F04217530738F0A90114
:1017E000DB019A01BD01DF01F801C1CFEF01F9CFA3
:1017F00090938B0580938A05CDCFFE01E20FF31FF6
:10180000819391932250310939832883D7CF209136
:10181000880530918905232B41F420911C023091D9
:101820001D02309389052093880520911A0230917A
:101830001B022115310541F42DB73EB740911E0220
:1018400050911F02241B350BE0918805F09189050A
:10185000E217F307A0F42E1B3F0B2817390778F087
:10186000AC014E5F5F4F2417350748F04E0F5F1FE6
:101870005093890540938805819391939FCFF0E021
:10188000E0E09CCFCF93DF930097E9F0FC01329723
:1018900013821282A0918A05B0918B05ED0130E090
:1018A00020E01097A1F420813181820F931F2091B5
:1018B0008805309189052817390709F061C0F09330
:1018C0008905E0938805DF91CF910895EA01CE174D
:1018D000DF07E8F54A815B819E0141155105B1F7AB
:1018E000E901FB83EA8349915991C40FD51FEC1795
:1018F000FD0761F4808191810296840F951FE901B3
:1019000099838883828193819B838A83F0E0E0E0DE
:1019100012968D919C9113970097B9F52D913C915A
:101920001197CD010296820F931F20918805309167
:1019300089052817390739F6309751F510928B052C
:1019400010928A05B0938905A0938805BCCFD383F4
:10195000C28340815181840F951FC817D90761F454
:101960004E5F5F4F88819981480F591F5183408393
:101970008A819B81938382832115310509F0B0CF41
:10198000F0938B05E0938A059ECFFD01DC01C0CF6B
:1019900013821282D7CF81E090E0F89400C0F894CF
:0219A000FFCF77
:1019A200FFFFFFFFFFFFFFFFFFFFFFFFFFFFFFFF45
:1019B200322E362E3200FFFFFFFF00008C05800022
:1019C200160018001A001C001E002000220024002D
:1019D200260028002C0017004C03190053031B009B
:1019E2005C031D00630321006A03230072032500C8
:1019F2007903290081032B0089032D0091032F0015
:101A0200990300000000CA04000000006503000002
:101A12000000C901340161011502920170018401C3
:101A22000000000084038103454E435F57686565EB
:101A32006C5F555000454E435F576865656C5F4467
:101A42004E005265616C53696D476561722D474660
:101A520043373030005265616C53696D476561727E
:101A62002D473130303050464431005265616C535D
:101A7200696D476561722D47313030304D464431D2
:101A820000232323235265616C53696D476561729C
:101A92002300454E435F414C545F555000454E4331
:101AA2005F4844475F444E00454E435F414C545F9C
:101AB200444E005265616C53696D476561722D47F2
:101AC2004D41333530003D310A003D300A00526548
:101AD200616C53696D476561722D474643353030FD
:101AE20000454E435F4844475F55500042544E5FA5
:101AF20056530042544E5F564E41560042544E5F7A
:101B020046440042544E5F59440042544E5F414C99
:101B1200540042544E5F41500042544E5F4941537B
:101B22000042544E5F4E41560042544E5F4C564C5A
:101B32000042544E5F4150520042544E5F48444767
:021B42000000A1
:00000001FF
